:02000000812855
:10000800A000030EA10083120508A3000F08A40096
:10001800A5012408A500A4010E08A4070318A50A31
:100028008E010E088F00A51B232801302502031C12
:100038002328031D2628F4302402031826283C20F0
:10004800A20A3228A51B32280B302502031C3228AD
:10005800031D3128B93024020318A201210E8300A0
:10006800A00E200E0B1009008312870185010800DD
:10007800220803195828013A03195B28033A03197F
:100088006028013A03196528073A03196A28013AD2
:1000980003196F28033A03197428013A03197928B8
:1000A8000F3A03197E2880288312051480288312AA
:1000B800051000008514802883128510000005159E
:1000C8008028831205110000071480288312071066
:1000D80000008714802883128710000007158028E5
:1000E80083120711000087158028831287110000EA
:1000F800071680288312071208008B0183168701D0
:100108008312871507309900F83083168500603010
:100118008100831290018316870196019615A2012A
:0E012800151638208B158B17831210149A2889
:02400E00D401DB
:00000001FF
